:100000008A010C2870287E289028A328AE28C028B2
:10001000F728072961296D2902208A110A12072071
:100020008A110A123C308312AB0006208A110A1290
:100030000E308312AB0006208A110A120A208A11A0
:100040000A1209208A110A12103083122502013087
:1000500003180301003C03196428A9080130031D9B
:100060000301003C0319632801308312A9000A3000
:100070002502013003180301003C03195128A00197
:100080002508303E0318A00AA6002608AA0004206E
:100090008A110A1283122608AC000B208A110A1258
:1000A00063288312A0012508373E0318A00AA60082
:1000B0002608AA0004208A110A1283122608AC001E
:1000C0000B208A110A12692883122908031969284A
:1000D000A9010A308312A20008208A110A122128DD
:1000E00083128501F8308316850006309F00831245
:1000F000051005118510831686010800FF30831650
:100100008600831285148312051100000515000076
:10011000861B8328051100008510831686010800C0
:100120008312851005102A08860003208A110A12FE
:10013000831205140515000005112D30A4000520BB
:100140008A110A120800A40CA40C3F30A405033045
:10015000A4020000A40BA928000008008312851047
:1001600005102B08860003208A110A128312051538
:10017000000005112D30A40005208A110A12080084
:100180003C308312AB0006208A110A12053083121C
:10019000A20008208A110A123C308312AB0006200C
:1001A0008A110A1205308312A20008208A110A124D
:1001B0003C308312AB0006208A110A1205308312EC
:1001C000A20008208A110A1208308312AB00062010
:1001D0008A110A1201308312AB0006208A110A121A
:1001E00006308312AB0006208A110A1208008E30F6
:1001F0008312A300000000000000000000000000C7
:10020000A30BFC280000A20BF72800000800F03028
:10021000831686008113831286010609A700A70EA4
:10022000A601831227080139FF390130031D003070
:10023000003C03192029270C7F39A700A60A1129A1
:10024000043083122602013003180301003C031915
:100250005D292608A8000F308316860081138312BB
:1002600086010609A700A601831227080139FF3974
:100270000130031D0030003C03194329270C7F394E
:10028000A700A60A3429043083122602013003187D
:100290000301003C031959292608A700A0012808DA
:1002A000A100A10D210DFC3927070318A00AA50004
:1002B0005C29FF308312A5006029FF308312A5005E
:1002C0000800193083169900A430980090308312EA
:1002D0009800BF3083168700080083122C0899000D
:0202E000080014
:00000001FF
